:0200000480007A
:100000006F000005732F2034930F80006308FF03F7
:10001000930F90006304FF03930FB0006300FF038E
:10002000130F000063040F0067000F00732F2034CC
:1000300063540F006F00400093E19153171F0000BD
:1000400023223FFC171F000023200FFC6FF01FFF2F
:100050009300000013010000930100001302000050
:100060009302000013030000930300001304000038
:100070009304000013050000930500001306000020
:100080009306000013070000930700001308000008
:10009000930800001309000093090000130A0000F0
:1000A000930A0000130B0000930B0000130C0000D8
:1000B000930C0000130D0000930D0000130E0000C0
:1000C000930E0000130F0000930F0000732540F102
:1000D0006310050097020000938202017390523072
:1000E000735044749702000093820201739052305F
:1000F00073500018970200009382020273905230EE
:10010000B70200809382F2FF7390023B9302F001EA
:100110007390023A7350403097020000938242017C
:100120007390523073502030735030309301000080
:1001300097020000938242ED739052301305100035
:100140001315F501634C05000F00F00F930110002B
:100150009308D0051305000073000000930200000F
:10016000638A020073905210B7B20000938292101B
:100170007390223073500030372500007320053013
:100180007350300097020000938242017390123442
:10019000732540F1730020309301200037050100E2
:1001A000130505C0530505F4531505E4930310002A
:1001B000631C750E9301300037C50000130505C0A0
:1001C000530505F4531505E493032000631E750CD5
:1001D00093014000378500001305F53F530505F4F2
:1001E000531505E4930340006310750C9301500010
:1001F00037850000530505F4531505E4930380008B
:100200006314750A9301600013050000530505F49B
:10021000531505E4930300016318750893017000FA
:100220001305F03F530505F4531505E4930300024D
:10023000631C75069301800037450000130505C057
:10024000530505F4531505E493030004631E750478
:100250009301900037850000130505C0530505F490
:10026000531505E493030008631075049301A0007F
:1002700037850000130515C0530505F4531505E433
:1002800093030010631275029301B00037850000DC
:10029000130505E0530505F4531505E49303002009
:1002A00063147500631030020F00F00F63800100CB
:1002B0009391110093E111009308D005138501007B
:1002C000730000000F00F00F930110009308D00599
:1002D0001305000073000000731000C00000000050
:1002E000000000000000000000000000000000000E
:0C02F00000000000000000000000000002
:1010000000000000000000000000000000000000E0
:1010100000000000000000000000000000000000D0
:1010200000000000000000000000000000000000C0
:1010300000000000000000000000000000000000B0
:081040000000000000000000A8
:040000058000000077
:00000001FF
